:020000040000FA
:02000000FA28DC
:08000800FF00030E8301A000BC
:100010000A08A1008A010408A200ED288A018207CB
:100020004B34503400341B344B34503400341B34C4
:100030004B34503400341B345F34363400341B34BA
:100040003F341B344B34503400341B345F3436346B
:1000500000341B343F341B344B34A1340034363469
:100060003234503400341B343234503400341B34B6
:100070003234503400341B342F34363400341B34C3
:100080003F341B345034503400341B345F34363426
:1000900000341B343F341B344B34A1340034363429
:1000A0002534503400341B344B34363400341B3484
:1000B0004B341B342534363400343634283436344B
:1000C00000341B342A341B342D341B342F341B349E
:1000D0002D3436340034363447341B3400341B346A
:1000E00035343634003436343834363400341B3446
:1000F0003C341B343F341B3443341B343F343634DC
:10010000003436345F341B3400341B3450343634FE
:10011000003436345F34363400341B3450341B34EE
:100120003F34503400341B344B34363400341B34E9
:100130003F341B343234A134003436342534503447
:1001400000341B344B34363400341B344B341B34F2
:1001500025343634003436342834363400341B34F5
:100160002A341B342D341B342F341B342D343634B5
:100170000034363447341B3400341B3435343634C1
:10018000003436343834363400341B343C341B34B9
:100190003F341B3443341B343F343634003436345C
:1001A0005F341B3400341B3450343634003436345E
:1001B0005F34363400341B343F341B344B345034FA
:1001C00000341B345F34363400341B343F341B346A
:1001D000003400340034003408000B1DF128C3251E
:1001E00059252208840021088A00200E8300FF0E72
:1001F0007F0E0900FF30A600FF30A70007309F00E8
:10020000A3262610E126A610E0262611DF26A61139
:10021000DE262612DD26A711D9262716D826A712F4
:10022000D7262717D626A717D5262816CC26281076
:10023000CE26FF30AA00FF30AB000930AC00061E0E
:100240002329A912C826AC0B1F29AB0B1D29AA0B09
:100250001B29A916C826A310B201B3012311A311AB
:10026000B801B90147263C08DF39502647263C082B
:10027000083850268B172312BA01FE30BD00BE018C
:10028000BF01C001C101C2018030C3008030C40081
:100290008030C500231724140130C600C701C801EF
:1002A000A410C9012415CA01CB011430CC00CD0122
:1002B0002A30CE00D001FF30D200D401D501143055
:1002C000D6001430D700D801D9014E08DA00013029
:1002D000DB000230E500BE266608CF000330E500F3
:1002E000BE266608D1000430E500BE266608D300AD
:1002F0000530E500BE266608CA000630E500BE26C9
:100300006608D7000730E500BE266608CB004A081D
:10031000013C031D8E292812CC2690292816CC26B4
:100320004B08013C031D9729A814CD269929A81034
:10033000CD264F25FF30E6008030E800FF30EA0090
:100340008030EC00FF30EE008030F0007623D423C4
:10035000231FAF29FF30D0003C08D200B429A41CD1
:10036000B329CA21B429C222FE23BE234008DF24B8
:100370007108C0004108DF247108C1004208DF2471
:100380007108C2004008C3004108C4004208C5000B
:10039000A629C929013046020318D0290630C60013
:1003A0004608063C0318D6290130C6004608013C21
:1003B000031DF729A31FE129013066235708BC005C
:1003C000A3133C08323C0318E629BC0100303C0270
:1003D0000318EC293230BC0057083C020319F429F9
:1003E0005708F30014309F253C08D700BF2A460861
:1003F000023C031D262AA31F062A4F08CE005108DF
:10040000D0005308D20002306623A3134D08013EEA
:100410003A02031D122A0530F30014309F250130E3
:10042000CA001C2A01304D023A02031D1C2A1E304C
:10043000F30014309F25CA014A08013C031D232AFA
:100440002812CC26252A2816CC26BF2A4608033C8B
:10045000031D552AA31F352A4F08CE005108D0008E
:100460005308D20003306623A3134D08013E3A021D
:10047000031D412A0530F30014309F250130CB00C5
:100480004B2A01304D023A02031D4B2A1E30F30065
:1004900014309F25CB014B08013C031D522AA814A0
:1004A000CD26542AA810CD26BF2A4608043C031D99
:1004B0007A2AA31F642A4F08CE005108D00053089F
:1004C000D20004306623A3134D08013E3A02031DF7
:1004D000702A0530F30014309F250130B025792AA9
:1004E00001304D023A02031D792A1E30F300143008
:1004F0009F25BF2A4608053C031D932AA31F892A6E
:10050000053066234F08CE005108D0000130BC00F2
:10051000A31355083C020318902AFF30D200912AF9
:10052000D201D50ABF2A4608063C031DBF2AA31FD5
:10053000A02A06306623BC018030CE00D001A31370
:10054000550854020318BD2AD80AD90A5808FF3C96
:10055000031DAC2AD901DB0A59080A3C031DB32A42
:100560005808D200B42AD20159080C3C031DBC2AF9
:100570005808D200D901BD2AD2013C08D5073A0853
:10058000CD000800013046020318C82A0430C60016
:100590004608043C0318CE2A0130C6004608013C38
:1005A000031DE22AA31FDD2A5108D0005308D20000
:1005B0004F08BC0001306623A3133C08CF004F084E
:1005C000CE00242B4608023C031DF62AA31FF12A65
:1005D0004F08CE005308D200023066235108BC00F9
:1005E000A3133C08D1005108D000242B4608033C3B
:1005F000031D0B2BA31F052B4F08CE005108D00065
:10060000033066235308BC00A3133C08D3005308EF
:10061000D2002523242B4608043C031D242BA31FB2
:100620001A2B043066235108D0000130BA00530859
:10063000D200A31303103A0CD40055085402031837
:10064000232BD501CE0AD50A08004608033C031D1A
:10065000632B4908013E3A02031D312BC70AC8012A
:10066000632B013049023A02031D632BC80A470875
:10067000053C03193D2BC701632B4808053C031DAE
:10068000632BC701C8012A30F30014309F250130C5
:1006900080262A30F30014309F25013080262A302E
:1006A000F30014309F25013080264B30F3001430C6
:1006B0009F25013080262A30F30014309F25013019
:1006C0008026C601A4143A08C9000800F100710888
:1006D000F200F208031D6D2B752B0730F300143068
:1006E0009F2501308026F203692B0800061ABB2BD8
:1006F000BE08031D7F2B231B7F2BC60AA3173E08B2
:10070000FE3C031DB92B0130BE00BF0A3F08013C6F
:10071000031DB42B231BA02B0530F30014309F25A1
:10072000013080261E30F30014309F2501308026D2
:100730000530F30014309F258030BC002317B42B04
:100740001E30F30014309F25013080260530F30061
:1007500014309F25013080261E30F30014309F2571
:1007600023130130C600A3173F08033C031DB92B18
:100770000E25BE0ABD2BBE01BF010800A31EC92B5A
:100780003B08643C0318C82B1E303B02BB00BC0A6C
:10079000D32B3B08643C0318D32B1E303B02BB0019
:1007A00001303C02BC000800861FE22B231AE12B1B
:1007B000061FE12BA3163D08BB00BA0ABC0AFF3096
:1007C000BD002316861BF42B231EF32B061FF32BD1
:1007D000A3123D08BB0001303A02BA0001303C02CE
:1007E000BC00FE30BD00231201303D02BD003D08BB
:1007F000003C031CFD2B0130BD0008005B08033CDE
:100800000318042C0130DB005B08013C031D262C7F
:10081000CE08031D192C5A08013C031D122C03306D
:10082000DB00182C5A08FF3C031D182C0230DB009B
:10083000252C4008F1004208F20041086C247108A0
:10084000C0007208C2007308C100692C5B08023C3A
:10085000031D482CCE08031D3B2C5A08013C031DE8
:10086000342C0130DB003A2C5A08FF3C031D3A2C93
:100870000330DB00472C4108F1004008F200420839
:100880006C247108C1007208C0007308C200692C92
:100890005B08033C031D692CCE08031D5D2C5A0820
:1008A000013C031D562C0230DB005C2C5A08FF3C37
:1008B000031D5C2C0130DB00692C4208F10041086B
:1008C000F20040086C247108C2007208C10073086D
:1008D000C0004E08DA000800F300FF30F1004E08B7
:1008E0007F3C031CA62C03104E0DFF3CF200DD01E3
:1008F000DE015008DC007208FF3CDF005F08B10039
:100900006008B0006108AF005C08AD005D08AC0095
:100910005E08AB000C263108DF003008E0002F082D
:10092000E1005F08B1006008B0006108AF00083066
:10093000F500A4113C263108DF003008E0002F0844
:10094000E1005F08F2075008F300DE2C80304E0211
:10095000F5000130F600EE267708F4007408F30085
:10096000DD01DE015008DC007308FF3CDF005F089A
:10097000B1006008B0006108AF005C08AD005D0820
:10098000AC005E08AB000C263108DF003008E00048
:100990002F08E1005F08B1006008B0006108AF00F7
:1009A0000830F500A4113C263108DF003008E000D3
:1009B0002F08E1005F08F3075008F2000800F1007B
:1009C000E401E301E101E0017108DF005208E20007
:1009D0005F08B1006008B0006108AF006208AD00B8
:1009E0006308AC006408AB000C263108DF00300857
:1009F000E0002F08E1005F08B1006008B000610866
:100A0000AF000830F500A4113C263108DF003008A3
:100A1000E0002F08E1005F08F1000800231F282DE7
:100A20000230F1004F08A8260330F1005108A82633
:100A30000430F1005308A8260530F1004A08A82622
:100A40000630F1005708A8260730F1004B08A82609
:100A5000C301C401C5010530F3000A309F250130F0
:100A600080260A30F3000A309F25013080260F309F
:100A7000F3000A309F25013080261430F3000A303D
:100A80009F25013080261930F3000A309F25013060
:100A900080261E30F3000A309F25A912C82E271089
:100AA000DC26A710DB262711DA268B168B170B11F5
:100AB000080080308100E50A65086602031D652D87
:100AC000E501E7014308E8006A2D67086802031999
:100AD0006A2DE70A2910670868020319702D291486
:100AE000CB26E90A69086A02031D7B2DE901EB01A7
:100AF0004408EC00802D6B086C020319802DEB0A72
:100B0000A9106B086C020319862DA914CA26ED0AD8
:100B10006D086E02031D912DED01EF014508F000F7
:100B2000962D6F0870020319962DEF0A29116F0890
:100B3000700203199C2D2915C9260B110800F40019
:100B4000B3017408B4007308B200A31423158B1604
:100B50000B1133083402031CAE2DA92D23110800FC
:100B6000F100B6017108B70023158B160B11013087
:100B7000B4002319BC2DC22D34083302031CC12D2F
:100B8000E725B92D080080308100231DE32DA31C2B
:100B9000DB2D01303902B900B908031DDB2D281007
:100BA000A31DD32D2814CE26A319D82DA315D92DD6
:100BB000A3113208B900B80AA6303802031CE22D8E
:100BC000B30AB801E52D2810CE260B11080037080E
:100BD000013C031DF92D3608F20006267208B60006
:100BE0007308B5003608F20006267208B6007308CE
:100BF000B400A310B5080319FE2DA3143508B200E4
:100C0000B301B408031D052E23110800F300720878
:100C10000E20F300F20A08002F08F5003008F60055
:100C20003108F7000030AF00B000B1001830F80014
:100C3000771C1B2E25260310AD0DAC0DAB0DF50C4E
:100C4000F60CF70CF80B182E0800262E2D2EB00FE0
:100C50000800AF0F0800AE0A08002D08B1070318FE
:100C600027262C08B007031829262B08AF070318DE
:100C70002B262A08AE0708000310A41D412E3118A8
:100C80000314AF0CB00CB10CF50B3C2E0800BE01E8
:100C90008130BF006B264008BD003D08BC00080045
:100CA000BA00BB018130BC003A08562EBD00831F3C
:100CB0005B2E23165C2E23123B1C602E8317612EA5
:100CC00083133C0884003D088000231E692E83178F
:100CD0006A2E83130800C000831F702E2316712E06
:100CE00023123E1C752E8317762E83133F08840033
:100CF0000008C000231E7E2E83177F2E831308005A
:100D0000F3007308F400F408031D872E8B2E643063
:100D10008C26F403832E0800F5007508F600F6080B
:100D2000031D932E972E32309826F6038F2E08003F
:100D3000F7007708F800F808031D9F2EA22E000088
:100D4000F8039B2E080003309F00E8261F13EB2EAC
:100D5000F2007108831603139B0083127208831636
:100D60009A001C158B1355309D00AA309D009C14D1
:100D70009C18B82E1C118B1783120800E60065081A
:100D8000831603139B001C141A088312E600080044
:100D9000CF2ECF2ECF2ECF2ED22ED22ED22E29082E
:100DA00086000800280885000800E22EE22EE22EC8
:100DB000E22EE22EE22EE22EE22EE52EE52EE52EAA
:100DC000E52EE52E270866000800260865000800C5
:100DD0008316031308008312031308007608003CEF
:100DE000031CF32EF92E0310F50D01307602F600E8
:080DF000EE2E7508F700080063
:02400E00223F4F
:00000001FF
